:020000040000FA
:04000000B3018F2990
:080008009529A50038088400C9
:100010003608F820841300052D1C36060319232802
:100020002508031D1B282B08FF3E031C24280A302B
:100030000F212B082428250AFF3003192328250B1C
:1000400023282C082428AE09AE0C8A29B316B31E27
:10005000B312B3192F28B315682003185628083097
:10006000A4007C20A30DA40B3128B31E61208620A0
:100070008220B31A56205B20230803108A29B31666
:10008000B31EB31233194928FE39B40033150310D7
:100090008A29331A5128A7003316682003185628D6
:1000A00027086F2003185628B31E8A29612086204E
:1000B00033113312B31138088400360884178004D2
:1000C00067283808840036098005841780050800F1
:1000D0005B208620612082203408B3190138A300F8
:1000E0000830A400A30D03185B20031C61208620A8
:1000F0008220A40B72285B208620380884003608F2
:100100000005FF3E39088400370964283908840057
:1001100037085E28A601A500B4172730A4001030C8
:100120009D200330A400E8309D20A40164309D2070
:10013000A4010A309D202508A828A3002608A200B3
:100140002508A10058212108031DB413B41B080081
:10015000303EA80085130513051383168513051378
:100160000513F030850583122808B318D4283A30D7
:10017000A200FC301D213330A700E9201030A2007E
:1001800068301D21E92064301C212230A700E920BD
:100190002830D3200C30D3200130D3200630D32098
:1001A000B3142808D4283314A700331CE2280513FD
:1001B000033C031CE728E7200730A200D0301D21B4
:1001C000031408003314FE3C03198A290517A70EEF
:1001D000331C33108517F030850527080F39850447
:1001E0008513A70E3318E92832301C2103140800A8
:1001F000841780048A2983161C141A0883169B0A04
:100200008A29030183169A001C1555309D00AA30D7
:100210009D009C149C180A291C119B0A8A29A40180
:10022000A300FF30A307031CA407031C8A29033083
:10023000A200DF301D211129A201E83EA100A20980
:10024000FC30031C2629A10703182329A1076400F9
:10025000A20F232921182C29A11C302900003029A4
:100260000800A30003303A29A30001303A29A30073
:1002700004303A29A90024082202031D4129230839
:100280002102043003180130031902302905031D2F
:10029000FF308A29A3002108A7002508A10027080C
:1002A000A5002208A7002608A2002708A6005A29B0
:1002B000A601A5011030A700220DA50DA60D23084B
:1002C000A5022408031C240FA60203186E29230884
:1002D000A50724080318240FA6070310A10DA20DDB
:1002E000A70B5C2921088A291030A900A201A101CD
:1002F000A80CA70C031C82292308A10724080318B3
:10030000240FA207A20CA10CA60CA50CA90B7829FE
:1003100025088A29831303138312640008008316B7
:100320000617861786168312082AA000030E83017B
:10033000BA000A08B500861B4F16861F4F12861B8F
:10034000CF16861FCF12861B4F17861F4F13861B93
:10035000CF17861FCF13061B4F14061F4F10061B07
:10036000CF14061FCF10061B4F15061F4F11061B7B
:10037000CF15061FCF1164004F0851020319002A40
:1003800064004F08003C031DD82964005008F03C6D
:10039000031DCE29CC010130CE00D62964005008BF
:1003A0000F3C031DD6290130CC00CE01D101002A1B
:1003B00064004F080F3C031DE0290F30D000002AD5
:1003C00064004F08F03C031DE829F030D000002AFB
:1003D00064004F08FF3C031D002A640050080F3CD6
:1003E000031DF629CC010130CE00FE29640050081F
:1003F000F03C031DFE290130CC00CE01FF30D100BE
:1004000035088A003A0E8300A00E200E0B1009005A
:1004100007309F00831681018312C230C900C330A8
:10042000CA000130A400F4301021FE30A9200130B0
:10043000A9205530A9206E30A9206930A9202D307F
:10044000A9205030A9204C30A9204C30A9202030C0
:10045000A9205630A9203330A9206130A920FE30D0
:10046000A920C030A9204430A9204C30A920313027
:10047000A9204D30A9204630A9204B30A92020309A
:10048000A9203030A9203930A9202F30A9203230BE
:10049000A9203030A9203130A9203030A920CC014A
:1004A000CE010130A400F430102183169B01831289
:1004B000FB20C500831601309B008312FB20C60081
:1004C000831602309B008312FB20D3008316033077
:1004D0009B008312FB20D2000630B8000230B60029
:1004E0000630B9001030B7004908412046084120C5
:1004F00045084120C2303F2088308B000630B800CC
:100500000230B6000630B9001030B700490841206B
:100510004608412045084120CE303F20EB232324CC
:1005200064004E08013C0319B92A64004C08013CE0
:100530000319CD2A6400861AA02A0A300F21E02A66
:100540000630B8000230B6000630B9001030B700EF
:100550004A0841202620CD00FE30A9208F30A92056
:1005600064004D1FB62A4C30A920B82A5830A92063
:10057000902ACE015208C5070318C60A4508A100F3
:100580004608A2007D30A40000303721031DCC2A8C
:10059000A030C5000F30C6009F2CCC015208C50208
:1005A000031CC6034508A1004608A2000F30A400A2
:1005B000A0303421031DDF2AC5017D30C6009F2CE9
:1005C000FE30A9200130A920FE30A9208030A920CA
:1005D0005E30A9202030A9205330A9207430A920F2
:1005E0006530A9207030A920FE30A920C030A92094
:1005F0007630A9202030A9207830A9202D30A920DC
:100600004D30A9206130A9206C30A92064004E082B
:10061000013C031D0D2BCE01852B64004C08013CD1
:10062000031D142BCC01242B0630B8002030B6005B
:10063000AD01FF30AB00AC010130AE004B0805202E
:10064000CB0003187E2A062BFE30A9200130A920FA
:10065000FE30A9208030A9204630A9206130A92091
:100660006B30A9207430A9206F30A9207230A920E6
:100670003A30A92064000A3053020318412B20307D
:10068000A920FE30A920C030A92053088A202D308F
:10069000A9206630A9206130A9206330A9206830E4
:1006A000A92064004E08013C03196B2B64004C0820
:1006B000013C0319752B0630B8002030B600AD019F
:1006C000FF30AB00AC010130AE004B080520CB0081
:1006D0000318E02A512BCE01D30A64000B305302D9
:1006E000031C742B0130D3007E2BCC01D303640098
:1006F0000130530203187E2B0A30D30083160230D8
:100700009B00831253080221242BFE30A9200130C4
:10071000A920FE30A9208030A9205330A9207430B0
:10072000A9206530A9207030A9203A30A920FE30D8
:10073000A920C030A9207D30A700A8015208A3003D
:10074000A4017421C7002608C8004808A60047086D
:100750008B206B30A9204830A9207A30A920640072
:100760004E08013C0319C92B64004C08013C0319D5
:10077000DA2B0630B8002030B600AD01FF30AB00F8
:10078000AC010130AE004B080520CB000318E02A75
:10079000AF2BCE015208A700A8010230A300A4018C
:1007A0007421D200640041305202031CD92B013065
:1007B000D200E42BCC010310D20C640001305202B1
:1007C0000318E42B4030D200831603309B008312C1
:1007D00052080221852B7D30A700A8015308A300F1
:1007E000A4017421BD002608BE004508A7004608E4
:1007F000A8003D08A3003E08A4007421BB00260801
:10080000BC000330A400E8304A21C1002208C20025
:100810004508A7004608A8005308A300A4017421B6
:10082000C3002608C4000730C3050030C4054308D0
:10083000A7004408A8007D30A300A4017421BF00D4
:100840002608C0000800FE30A9200130A920FE3093
:10085000A9208030A9204108A1004208A200273029
:10086000A40010303121031D432C2030A920410861
:10087000A1004208A2000330A400E8303121031D8A
:10088000432C2030A9204208A60041088B202E309E
:10089000A9203F08A1004008A200A4016430312132
:1008A000031D5F2C3030A9203F08A1004008A200A2
:1008B000A4010A303121031D5F2C3030A9204008EB
:1008C000A6003F088B202030A9204D30A9204830B9
:1008D000A9207A30A9202030A920FE30A920C030DC
:1008E000A9205330A9207430A9206530A920703088
:1008F000A9202030A9207D30A700A8015208A3001C
:10090000A4017421BD002608BE003D08A7003E08D2
:10091000A8005308A300A4017421BD002608BE004E
:100920003E08A6003D088B202030A9206B30A9206E
:100930004830A9207A30A9202030A9200800831649
:100940009B01831245080221831601309B0083120C
:06095000460802217E2A88
:02400E00383F39
:0842000000002800010001008C
:00000001FF
